:100000007590FF75B0FF7D007E00758130D220D2E3
:1000100021C223D222C224C2D3C2D4740075F001FB
:10002000312631FE74A0513A401D7400513A31FE20
:1000300074A1513A5116510D20B40751BCD224027B
:10004000025CB46402D223740A75F01431267E0077
:10005000302412EE600F741975F032312631B8D2A7
:10006000227E0080D67E007B0031390BBB5002809F
:10007000DF60F67B00318B9002D493FF2023089041
:1000800002CDEE9302009B31FE74A0513AEE045172
:100090003A31FE74A1513A5116510DC394306F0E8E
:1000A00070AE202305EE930200BE31FE74A0513ADB
:1000B000EE04513A31FE74A1513A5116510DB4FF7C
:1000C0006330240D51AB741E75F0193126319A80BE
:1000D000FE741E75F019312620B337319AC2B7C2AB
:1000E00020740AC39404F8743775F0233126C221B2
:1000F000318BD221D8F17803743775F02331263152
:100100008BD8F5743775F01E312631A9D2B7D220BD
:100110000150302005319A02011C31A9B220A220E1
:1001200092B701500169D2D4A8F0F97AFFDAFED96A
:10013000FAD8F775F001C2D4227A0079007FFE8FD9
:1001400090A89074053126E590FC6870F474053130
:1001500026A890EC6870EAECF45470600AB90024A8
:1001600023093350FC701DE97004EA2403FAEF23DD
:1001700030E405FFF59080C9E96009C32AFC6D6091
:1001800007ECFD227400FD22740022755901755B95
:100190000F755A0A75584B31C722755903755B0F95
:1001A000755A0A75584B31C722755901755B96759A
:1001B0005A0175584B31C722755903755B96755AAC
:1001C0001475584B31C722D2D3AB59A95B7F0AA80B
:1001D00058D8FEC2B5A858D8FE302102D2B5DFEFFC
:1001E000D9EBD2B5BB01030201F6AA5A7E0F7F00FC
:1001F000DFFEDEFADAF6DBD3C2D322000022D2B170
:10020000D2B031FBC2B131FBC2B031FB22D2B0312E
:10021000FBD2B131FB227808D2B131FBD2B031FB35
:10022000A2B1C2B031FB33D8F3D2B131FBD2B0317D
:10023000FBC2B031FBC2B131FB2278083392B1313D
:10024000FBD2B031FBC2B031FBD8F1D2B131FBD21D
:10025000B031FBA2B1C2B031FBC2B1223139202290
:10026000070BBB500302029060F2BEFE0302029035
:100270009002D4932430C0E07B00318BC2220E3137
:10028000FE74A0513AEE513AD0E0513A510D80CC73
:100290000E31FE74A0513AEE513A74FF513A510DAD
:1002A000740A75F0143126319A014531FE74A0515B
:1002B0003A7400513A7464513A510D2231FE74A0DF
:1002C000513A7400513A74FF513A510D2235353587
:1002D000383233FFFAF300FA030201060504090875
:0102E0000716
:00000001FF
